:1060AD0033302E322020200002000205020B021098
:1060BD000216021C02220228022E0234023A02406B
:1060CD000247024D0253025A02600267026E0274C9
:1060DD00027B0282028902900297029F02A602AD04
:1060ED0002B502BC02C402CC02D402DB02E302EB15
:1060FD0002F402FC0304030D0315031E0326032FF4
:10610D0003380341034A0353035D0366036F0379A9
:10611D000383038C039603A003AB03B503BF03CA2C
:10612D0003D403DF03EA03F4FFFF064003200190CD
:10613D00010A00C8008500640050003500280020C9
:02614D00001A36
:1051A8004105B0054304200105B14304230105B1BD
:1051B8004106B200C1074106B1004204AE000041F9
:1051C800042600C1034104940041041C0041045713
:1051D80000C104C102C101C10CC105C106C1094118
:1051E800042F00C10DC100C10A41049100410452BD
:1051F8000041041B004204AA000042049900004236
:10520800049200004404A000000000410455F0424C
:1052180004950000C1084404A60000000041049859
:10522800004104590041045800420453000041045D
:10523800A55B410434AA4104A4AA41044F004204D6
:1052480050000041049BFF41048FFF410435FF419A
:105258000456004404300800000044049C04F1BBD8
:10526800CD4404270000000044041400000000445A
:10527800042B0000000044040E000000004204ACAF
:105288002EE04204120000C18B43045A31323041EF
:0A52980004900044040A000014CB47
:1050360074362FF582E43404F583229008DFE025E8
:10504600E024C7F582E43406F583E0FEA3E0FF9092
:1050560008E0E025E0245DF582E43404F583EEF013
:10506600A3EFF09008E0E004F0229007F91244ED77
:105076009000051241CBFF9000061241CBFD900037
:10508600040241CBEF25E024B8F582E43406F5832B
:105096002290082C12445D90082C0244459007F992
:1050A6007B017A0779E60244ED9008DFE0FFC394BE
:1050B6001922EF25E024C7F582E43406229008DFA2
:1050C600E004F02290041D7B017A0479B00244EDDD
:1050D600E025E02435F582E43461F583E493FE743B
:1050E600019322FFE43EFEE43DFDE43CFC02445D08
:1050F6007FFF7EFF7D0F7C009004A0024451E4FCFC
:10510600FDFE1244510242DAEF25E0245DF582E409
:1051160034042290082812445D90082802444574FD
:10512600F92FF582E43406F58322E02FFFC364806D
:105136009480229000031241CBFF9004A5E06F22D9
:105146009004A0024445E475F001024293124451D2
:10515600C302440D9008E0F0A3F09008DFF022901F
:10516600041D0244B67C007D0CAE0202423EED54A4
:105176003FF0EDAE047806223395E08DF0124293AF
:10518600D3227B017A0579B10244EDE475F0011270
:1051960044D67401229006B6E064012290041402FB
:0251A60044457E
:106EAE00125165C003C002C0019004181244B6D03E
:106EBE0082D083D0E06B7008E965827003EA658347
:086ECE0060037F01227F002216
:106F24001251651241B2FF90041E12514C12516568
:106F340074019005B06B7008E965827003EA65839B
:056F440070031250CAA9
:016F49002225
:05761C00C205D20622A8
:106A95009006B6E0FF900459F0B4010A9006B6746A
:106AA50002F0C20D8014EFB402089006B67401F02E
:106AB5008008EF70059006B604F0900459E0B40123
:106AC5000A9006B6E0B4020312761C200609900669
:0D6AD500B6E0B40202E4F012501B024C4A7D
:084FBE009006B5E064017036B5
:104FC6009006C5E0FAA3E0FBFF12516B900915EFBE
:104FD600F0AF0312516BAF05A3EFF0C3940690092F
:104FE60015E05002800204F075F00CA4FF9006C58F
:064FF600E5F0F0A3EFF06E
:104FFC009006B5E004F0D394024002E4F012501B8A
:03500C00024C4A09
:1071BF00200809A203B39203D208800CC203C203B2
:0B71CF00127579E4900498F0024C4A1D
:1067CE00900498E06023900426E0FF700404F080AB
:1067DE0038EFB401089004267402F0802CEF6402A6
:1067EE00702790042604F08020900426E0FF7004A9
:1067FE0004F08015EFB40107E4900426F0800AEF50
:10680E00B402069004267401F0900426E07005C2CE
:0F681E00031275799006B6E0700204F0024C4A3E
:106E5B00D39006C6E094009006C5E09400401890CD
:106E6B0006B5E09006C5B4020774FF75F0F4800414
:0A6E7B0074FFF5F012429302501B61
:106E8500C39006C6E094549006C5E0940050179050
:106E950006B5E09006C5B40206E475F00C8004E47E
:096EA50075F00112429302501B2A
:1056CB00900819E0FEA3E0FFE4FCFD9008301244C3
:1056DB005D9006C3E0FEA3E0FFE42FFFEE34F8FE7F
:1056EB00E434FFFDE434FFFC9008301251089008BD
:1056FB003412445D900834124445E4FB7A08F9F8FF
:10570B00126B7590083412445D9006C6E02418FFA6
:10571B009006C5E03400FE7C007DC312422C30099C
:10572B000874482FFF74123EFEEF7802CEC313CEDF
:10573B0013D8F9FFE4FCFD125119900834124451AF
:10574B001242BF125119EC33500A900828124469C7
:10575B0000000000E47F917E14FDFC9008281244A9
:10576B0051D31243F7400A900828124469000014E1
:10577B009112511F125097E47B207A01F9F81242D3
:10578B00DA125097E47B917A14F9F81243651250B0
:10579B0097EF241A90082C1250E9E47B40FAF9F8A1
:1057AB0012509D124365AB0712509DEF543FFFC340
:1057BB0074049BFEEF25E024B5F582E43460F58399
:1057CB00E493FD7401939004AECDF0A3EDF0AF061E
:1057DB009004AEE0FEA3E0A807088005CEC313CE6D
:0957EB0013D8F9F0EE9004AEF0C1
:0157F4002292
:0A7579007F19900436E4F0A3DFFC54
:0175830022E5
:03501500027579A8
:10740C00E4D39F500DEFC394045007EF2498FF1260
:03741C006B2D22B3
:046C7D00AD07AC06AD
:106C8100ED4C70079005B0E02407F09009181251FF
:106C910074CEA2E713CE13D8F8FDAC06543F900989
:106CA10017F07F97126B2D900918E0FF126B2D9052
:076CB1000917E0FF026B2D43
:10743200900929EFF07F94126B2D900929E0FF0249
:027442006B2DB0
:107130009006C0E004F0C394044002E4F09006C05E
:0D714000E0FF12740C7FE9126B2D02501B52
:1070F0009006C0E0600414F080069006C07403F0AF
:107100009006C0E0FF12740C7FE9126B2D02501B39
:1071F50090092AEFF0BF1A051271BF800A90092A7B
:0A720500E0B41903126A95024C4A26
:1062860090092BEFF064196004E0B41A0890092B0A
:10629600E0FF0271F530033590092BE0FFD3941827
:1062A60050047E0180027E00E4D39F50047F01806B
:1062B600027F00EF5E600B90092BE0243612503906
:1062C600E4F012750FEF704CC203024C4A9004269C
:1062D600E06402603F90092BE0FFD3941850047EDF
:1062E6000180027E00E4D39F50047F0180027F007C
:1062F600EF5E602090092BE0FF64116017EF6412D7
:106306006012125125E0600C90092BE024361250E1
:05631600397401F022C2
:106ED600900426E07020EFD3941850047E018002BF
:106EE6007E00E4D39F50047D0180027D00ED5E604C
:076EF60005125036E4F02202
:0D753A00900497E0C394185003E004F02281
:0975D000900497E0600214F0221F
:10734200E4D39F5012EFC39419500C125125EDF063
:087352007005125036E4F02230
:056CF200900909EFF01C
:106CF70090090B125174CEC313CE13D8F9FDAC060D
:106D0700543F90090AF07F90126B2D900909E0FF1C
:106D1700126B2D90090BE0FF126B2D90090AE0FF13
:036D2700026B2DCF
:10714D00900919EFF0A3EDF07F95126B2D900919B1
:0D715D00E0FF126B2D90091AE0FF026B2D70
:1074D0001250B8F583ECF0A3EDF0126CF202501BE1
:1074440090092CEFF07F8C126B2D90092CE0FF0239
:027454006B2D9E
:1074560090092DEFF07F8D126B2D90092DE0FF0224
:027466006B2D8C
:05631B00E49008EAF027
:106320009008EAE0FF1250B9F583E0FCA3E0FD908D
:1063300008EBECF0A3EDF0126CF29008EAE0FF2419
:09634000F9125128E0FD12714D23
:106349009008EAE004F0E0C3941940CBE49008E92E
:10635900F09008E9E0FFC39404501A12740C9008F5
:10636900E9E012508BE0FEA3E0FF126C7D9008E992
:10637900E004F080DC9006C0E0FF9008E9F01274B8
:106389000C9006B7E0FF1274329006C1E0FF127458
:0E639900449006C2E0FF1274567FE9126B2D8D
:0163A70022D3
:0C756100EF6003D38001C39201024C4A8A
:1073F8007406D39F5009EF94075004D20C8002C240
:047408000C024C4ADC
:0A69EF00E4D39F504EEF9419504975
:1069F9001250B8F583E0FBA3E090091BCBF0A3EBA1
:106A0900F0ED90091B12517E90091CE094C6900983
:106A19001BE06480948340077403F0A374C6F0C339
:106A290090091BE0648094805004E4F0A3F090097D
:096A39001BE0FCA3E0FD1274D087
:016A42002231
:0B7584009006B7EFF012743202501BAB
:10720F009006B71251305002E4FFD3EF648094849C
:0A721F0040027F0412758402501B28
:0B758F009006C1EFF012744402501B84
:0B759A009006C2EFF012745602501B66
:107229009006C11251305002E4FFD3EF6480948C70
:0A72390040027F0C12758F02501BFB
:107243009006C21251305002E4FFD3EF6480948C55
:0A72530040027F0C12759A02501BD6
:1045750075FFDE75FFAD1272AB9007D2124469006C
:104585007C9D0A9007D612446900000FA09007DAB7
:10459500124469000007F99007DE1244690000F82B
:1045A50007125015126E0212718712716A12700687
:1045B50012749D1274681274E01275E912747A12FD
:1045C50075009007E212446905D75C8043A8204333
:1045D500A81075E60875E7069004A5E0FF12754773
:1045E50043F602D2AF124C4AD2857E017F00900578
:1045F500B174AAF0A3DFFCDEFA7E017F001250CA77
:104605009004181244EDE49006B3F01270CF126EC8
:10461500FDEF606A126AE2EF1244F6464201464730
:1046250002465C03466104466605464C06466B0732
:10463500467508467009467A0A0000467D126A9555
:104645008036124FBE80319004A5E0FF7BFF7A6073
:1046550079AD1269418021127130801C1271BF80C1
:10466500171267CE801212708D800D126E5B800856
:10467500126E8580031275FE126EFDEF7096126E36
:09468500AEEF640160030247FE80
:10468E00126F24900802EFF020E703024750E090EB
:10469E000455F01244F646E48946E88A472CA847AA
:1046AE0030A94734AA4738AB473CAC4740AD4744E6
:1046BE00AE4748AF4724B24720B346FCB44700B5D7
:1046CE004708B6470CB74714B84718B946F0BA466C
:1046DE00F6BC000047FE7F018002E4FF1275610206
:1046EE0047FE1275BB0247FE12631B0247FE7F0197
:1046FE0080027FFF12720F0247FE7F0180027FFF52
:10470E001272290247FE7F0180027FFF127243025E
:10471E0047FE7FFF80027F011271DA0247FE7F01A2
:10472E00801A7F1080167F4080127F7F800E7FFF61
:10473E00800A7FF080067FC080027F8112688A0225
:10474E0047FE900455E01244F6478282478C834719
:10475E00E18B47EB8E47F48F4796A0479FA147A862
:10476E00A247B1A347BAA447C3A547CCA647D5A72E
:10477E00000047FE900802E0FF12628680729008E9
:10478E0002E0FF126ED68068900802E0FF7D018085
:10479E003D900802E0FF7D108034900802E0FF7D1E
:1047AE0040802B900802E0FF7D7F8022900802E07F
:1047BE00FF7DFF8019900802E0FF7DF080109008C9
:1047CE0002E0FF7DC08007900802E0FF7D81126944
:1047DE00EF801D900802E0FF1273F880139008021C
:1047EE00E0FFE4FD8007900802E0FF7D01127342B6
:1047FE00300A0A9004A5E0FF1272F7C20A7B017A12
:10480E000779E612704AEF70030249349007E8E028
:10481E001244F6487C04489005484C14484016480B
:10482E00441748511A48651B48701D48761E0000F3
:10483E0048ADD2018002C201124C4A0248ADD202EA
:10484E000248AD9007F61250A61241B2FE9004A592
:10485E00E0FF6E704A80059004A5E0FF1273890296
:10486E0048AD1275F70248AD1276160248AD1250D9
:10487E00A3125139702930011E125070FB1266F9C5
:10488E0080151250A3125139701530010A12507052
:10489E00FB1264B51270CF9004A5E0FF12731020C6
:1048AE00010302480B9007E8E014603014602024E6
:1048BE00FB603514605924F9600302480B7B017AC2
:1048CE000779E69007FF1244ED1270AE02480B1204
:1048DE0049429006B3F01275BB02492E124942901E
:1048EE0006B3F01270CF8038124958125084FD90E2
:1048FE0000051241CBFBC0039007FC1244B690009A
:10490E00061241CB900847F0D0031261EF801112CE
:10491E004958125084FD9000051241CBFB12591FCD
:10492E001275A502480B20000302461312631BC228
:04493E00000246131A
:104942001274AE7B017A0779E69007F61244ED9075
:1049520000031241CB221274AE7B017A0779E690F2
:0D49620007FC1244ED9000031241CBFF2230
:10748C0012508AECF0A3EDF0AE04FF126C7D0250AA
:01749C001BD4
:10688A009006C0E0FEE4D39E5051EEC39404504BF0
:10689A00EE12508BE0FDA3E090091DCDF0A3EDF0C0
:1068AA00EFFD90091D12517E90091EE094F49009A3
:1068BA001DE06480948140077401F0A374F4F0C36E
:1068CA0090091DE0648094805004E4F0A3F0AF06C0
:0B68DA0090091DE0FCA3E0FD12748C8F
:0168E5002290
:0E751E009006C0EFF012740C12501B024C4A83
:1071DA009006C0E02FFFD36480F8748098500BC3E8
:0A71EA00EF64809484500312751EB8
:0171F4002278
:0675FE00A209B39209226C
:1074E000E4F58475D84075D98375DA3175DB3122BE
:0775E900E4F58475D10322D3
:10700600AF8475840F75A43475A5FC75A6FF75A7A6
:10701600FF75E11775E340E4F59075A0FFF5B08FB5
:0170260084E5
:017027002246
:10718700AF84E4F58475C9E775CBF875CA0785CB75
:0B719700CD85CACC75C804D2AD8F8432
:0171A20022CA
:10716A00AF8475840275C9E775CB6075CA7F85CA15
:0C717A00CC85CBCD75C80443E7048F849E
:0171860022E6
:1072C500AF84E4F584758920758E10758D40F58B36
:0872D5004388408F8443A88028
:0172DD00228E
:10749D001272C5E4F584759850F584D2AC43A810EA
:0174AD0022BC
:10746800E4F584759A4075F809759D01759D10C2FB
:02747800FA22F6
:106B2D009006B2E07002740160F6C2AC900420E4ED
:106B3D0075F0011244BFEF1241F89004201244B6D3
:106B4D0074019006B16B7008E965827003EA658384
:106B5D0070069004201251889006B2E004F02007D0
:086B6D0004D207D299D2AC2238
:03500F00025C56EA
:105C5600C0E0C0F0C083C082C0D075D000C000C014
:105C660001C002C00375840030982FC298900418B2
:105C76001244B6E5991241F8900418125191900514
:105C8600B06B7008E965827003EA6583700690045C
:105C9600181250CD9006B1E004F030996F9006B21C
:035CA600E0606556
:105CA9009004231244B61241B290092EF0C29924ED
:105CB900EC601214601714601C2488701E9005B0E3
:105CC900740BF080169005B07407F0800E9005B043
:105CD9007405F080069005B07403F090092EE0F584
:105CE900999006B2E014F09004231251919006B1F4
:105CF9006B7008E965827003EA6583700C90042370
:035D0900125188AC
:105D0C008004C299C207D003D002D001D000D0D0F9
:095D1C00D082D083D0F0D0E03237
:10706C00C2069004A012446900000000E49004924F
:10707C00F0A3F0900426F09006B6F0127579024C4D
:01708C004AB9
:1064330030053A9006C1E0700280281250F6C3126C
:1064430043F750291250FE9006C11250D6FFE4FCC8
:10645300FD1242BF9004A012445D1250F6D31243C2
:10646300F7400A9004A0124469000FFFFF30063181
:10647300125146EC33402A125146C006C00790061B
:10648300C21250D6FBAA06E4F9F8D007D00612428E
:10649300CC9004A012445D125146EC3350031270A9
:1064A3006C1251467804124431900492EEF0A3EF3B
:0264B300F022D5
:03501200025DF448
:105DF400C0E0C0F0C083C082C0D075D000C000C075
:105E040001C002C003C004C005C006C007C2CF3031
:105E1400082CE47FD07E07FDFC9004A61251535059
:105E2400119004A6124445EF24019004A61250E9EF
:105E3400800CC2089004A61244690000000090047B
:105E440050E0FEA3E0FFEE702FEF14600C14600E20
:105E5400240270241275F0801F125594801A126463
:105E640033900457E0601190041CE0600414F08047
:105E740007D20A900457E4F090045012514CFEC328
:105E8400E5F09403EE648094804007900450E4F0BD
:105E9400A3F01256CB124C4AD007D006D005D0043A
:105EA400D003D002D001D000D0D0D082D083D0F0A3
:035EB400D0E03209
:106F4A00200D17D20DD205E4900492F0A3F090041C
:106F5A00A012446900000000C2067F3290045D74EA
:056F6A00FFF0A3DFFCB5
:016F6F0022FF
:1073E30012519B6002C2057F3290045D74FFF0A3CB
:0573F300DFFC027579CA
:1068E60090092FEFF090049C125104900427124453
:1068F6005D90092FE0FF90043012510490040E12AF
:10690600445D1251A29004271244511242BF801ACC
:1069160090040E124445900414125153401412511F
:10692600A290040E1244511242CC90041412445DFB
:0B69360080DE1251A2781B12441E22CA
:10496F00900498E0900456F0E4900498F09008DFDB
:10497F00F01250AF5013125036E060089004987444
:10498F0001F080051250C380E8900456E070099042
:10499F000498E06003126F4A900498E070047F015E
:1049AF0080027F00900456E05F60031273E390046F
:1049BF0098E07003024C1E90049BE030E727E490D0
:1049CF0008DFF01250AF501D125036E06012900603
:1049DF00B7E06404600F9008DFE090049BF080055F
:1049EF001250C380DEE49008DFF01250AF50151262
:1049FF005036E0600A9008DFE090048FF0800512D7
:104A0F0050C380E69008DF7418F09008DFE0601A5A
:104A1F002436125039E0600A9008DFE0900435F038
:104A2F0080089008DFE014F080E09006B7E064049F
:024A3F00703CC9
:104A410012515A1250AF5012125036E060071250F4
:104A510041A3E004F01250C380E99008E0E0FFC3F5
:104A61009419500D12510EF583E4F0A31250688091
:0C4A7100E99008E1E0FF1268E6024ACD7F
:084A7D009006B7E064037053DA
:104A850012515A1250AF5012125036E060071250B0
:104A950041A3E004F01250C380E99008E0E0FFC3B1
:104AA5009419500D12510EF583E4F0A3125068804D
:104AB500E9126D2A9008E2EEF0A3EFF09008E1E02C
:104AC500FD7C0012423EAF0590049BEFF012510FA2
:034AD500024BABE6
:104AD8009006B7E0FF7006900923F0800AEFB40152
:104AE800069009237401F0900923E0FF70369008BE
:104AF800DFF090049BE004F0E0B41902E4F09008C1
:104B0800DFE0C39419505D90049BE02436125039BD
:104B1800E070511250C390049BE004F0E0B419DE39
:104B2800E4F080DAEF6401703B9008DFF090049BBA
:104B3800E0600414F0800590049B80239008DFE077
:104B4800C39419501F90049BE0FF2436125039E09B
:104B580070121250C3EF90049B600414F080DD744F
:104B680018F080D89006B7E064027030900923E00E
:104B7800FF7014900435E0FE90049BE0B5060890A1
:104B880009237401F08015EFB4011190048FE0FF40
:104B980090049BE0B50705E4900923F090049BE09E
:104BA8001250B9F583E0FFA3E0900499CFF0A3EF8A
:104BB800F09006C0E0FF9008DFF0900499E0FCA3B5
:104BC800E0FD12508AE0FEA3E02DFDEE3CFC7406E9
:104BD8002DFD74FF3CFCC3648094805003E4FCFD0D
:104BE800D3ED94C6EC6480948340047C037DC6AF07
:104BF80005900499ECF0A3EFF0900499E0FEA3E08F
:104C08007806C333CE33CED8F9F0EE900499F0A3EA
:104C1800E054F0F0800690049B74FFF0E490049157
:104C2800F090041BF0900498E07003300613E490B1
:104C3800042FF090049104F0900452F090041B04A7
:014C4800F07B
:014C49002248
:03503300025EB763
:105EB700C0E0C0F0C083C082C0D075D000C000C0B1
:105EC70001C002C003C004C005C006C007C2CFC3DB
:105ED700900413E094E8900412E0940350161251D2
:105EE7004C900412E07004A3E064C87007300B0400
:105EF700C20BD20012519B6011900426E0FF64018F
:105F07006008EF640260033006369006B5E0703033
:105F17009004AEE0FEA3E0FFC39004ADE09FFF90C6
:105F270004ACE09EFEF0A3EFF0D39400EE648094FF
:105F370080500D12496F9004AC742EF0A374E0F0FA
:105F4700D007D006D005D004D003D002D001D000AE
:0B5F5700D0D0D082D083D0F0D0E03258
:10708D0012519B6011900426E0FF64016008EF64CB
:10709D0002600330060A9006B5E0B4010312496F91
:0170AD0022C0
:0775F000E4F58443E81022DA
:1055940090042FE004F0C394034002E4F090042F3D
:1055A400E0FF245AF582E43404F583E09008AAF07D
:1055B400EF14605314700302563B24026003025636
:1055C40088900499E0FEA3E0FF7C007D6412451CF2
:1055D400E47B6AFAF9F81243659008AD12445D90D1
:1055E40004041244459008AD12515370030256CA84
:1055F4009008AD12444590040412445D9008AD1225
:105604004445AC06EF8029900402E0FEA3E0FF903D
:105614000492E0FCA3E06F7002EC6E70030256CAC1
:10562400900492E0FEA3E0FF900402EEF0A3EFF0FA
:105634009008ACF0EC8049900452E0600414F080CF
:1056440013900491E0600614F074FF8001E4900468
:10565400AAF0A3F090041BE0600214F09004AAE006
:10566400FEA3E0FF900408E06E7003A3E06F6056B1
:10567400900408EEF0A3EFF09008ACF09004AAE0D8
:105684009008ABF0E4F584C2FAFF0FEFB464FBE5D5
:105694009A20E7FBE4F59BE59A20E7FB9008AAE053
:1056A400F59BE59A20E7FB9008ABE0F59BE59A2093
:1056B400E7FB9008ACE0F59BE59A20E7FBE4FF0FDD
:0656C400EFB464FBD2FA12
:0156CA0022BD
:106D2A007F217EF17D7D7C0090040A125108EF24B8
:106D3A00F3FFEE3490FEED3424FDE43CFC90040AAB
:106D4A0012445DE47BFF7A7FF9F890040A12444505
:076D5A00124365AE02AF0316
:016D6100220F
:106FBC00E0FEA3E0A60608F6E4F584C2AF43B701F1
:106FCC0022E475F0011242A985F082F58322EEF0DD
:056FDC00A3EFF0A32269
:106D9A00AB84A2AF9216E4FCFDED9008ED12445DBF
:106DAA009008EF780C126FBC438F02438F0118E6EC
:106DBA00FE08E6F5828E83E4F053B7FEF58FA2163D
:066DCA0092AFAF038F84BD
:016DD00022A0
:026BFC00AB05E7
:106BFE00AA84A2AF9217E4FCFDED9008F112445D59
:106C0E00EBFF3395E0FEEFF44E601C9008F3780E28
:106C1E00126FBC758F0118E6FC08E6F5828C83EBCB
:0F6C2E00F053B7FEE4F58FA21792AFAF028F8439
:016C3D002234
:106A43009008CD126FDAECF0A3EDF0A3EAF0A3EB1C
:106A5300F09008D1E07002A3E060369008CDE0FE2C
:106A6300A3E0FFA3E0FCA3E0F5828C83E0FD126BBF
:106A7300FC9008D174FFF5F01242939008CFE475AF
:106A8300F0011242939008CDE475F0011242938015
:026A9300C0221F
:0875D900E4900000F0A3F02291
:106F7000900000E0FEA3E0FF126D9A900000E0FE9A
:106F8000A3E0FF7C007D027B007A04126A43E49058
:066F90000000F0A3F02256
:0A653000A9059008D3EEF0A3EFF0E8
:10653A00EE54FCFE900000E0FCA3E0FD7002EE6C5D
:10654A006042ED4C6003126F709008D3E0FEEE5487
:10655A00FCFE7F00900000F0A3EFF09008D5126FC8
:10656A00DA7400F0A37402F07E049008D5126FCD9D
:10657A00E493FD9008D7126FCDEDF0EF1F70011E66
:10658A00EF4E70E69008D3E0FCA3E0FDEC5403FC68
:0C659A0074022DF58274003CF583E9F0DA
:0165A60022D2
:106D62009008B1126FDA1244ED9008B674FFF5F094
:106D72001242A945F060209008B1E475F001124278
:106D8200A9AFF0FE9008B3E475F0011244BF1241BE
:086D9200B2FD12653080D2222F
:1052A2004207D0000042077B00004207760000C19F
:0552B20010C10FC10E48
:106CB800900771E475F001024293D39007D1E094F4
:106CC800009007D0E06480948022E0FEA3E0247D59
:106CD800F582740722900776F0A3F02274FFF5F08E
:0A6CE800024293FCE5F064404C22E8
:0A75C600C20FC210E490077AF02211
:10711000E49007D0F0A3F090077BF0A3F0A3F01267
:107120006CDD900771F0A37440F0E4900779F022D1
:067604001275C6027110B0
:1072DE00E4F5848FC343C30175C04475CF8EC2C31A
:0972EE0043E60290077804F02247
:1074AE00E4F58420C7FDC2C2127604E4900778F09A
:0174BE0022AB
:0B75A500E4F584D2C290077804F022C5
:0D754700AE071272DE900775EFF0027604B9
:106FE100E490091FF0A3F0300F02FF222010FDD220
:106FF1000F900773E4F0A37410F09007BEEFF0E474
:04700100A3F07F0178
:017005002268
:106E2F00300F0A900773E07002A3E070037F002217
:106E3F00900773126CE49007BFE0FE04F074C02E4D
:0C6E4F00F582E43407F583EFF07F0122A8
:0B75B000300F07C20FD2101250212232
:0E502100AF84E4F58420C7FDC2C4D2C58F84DD
:01502F00225E
:10661D009008B91244ED900778E07002FF229008BF
:10662D00BCE0FE6005D3941040037F0022126FE1A1
:03663D00EF6049C2
:10664000E49008BEF09008BCE0FF9008BEE0FEC3F6
:106650009F501F9008B91244B68E82758300124174
:10666000CBFF126E2FEF7002FF229008BEE004F005
:1066700080D3E490077AF01275B09008BDE0700303
:096680002010FD90077AE0FF22D2
:036689007FFF226E
:0B6009009008F51244ED9008F8EDF04F
:10601400E4FF126CC250012253E6FD900776126C25
:10602400D23EF583E0FF900776126CBB126CEB70E6
:1060340003126CDD126CB8E4FE9008F8E0FDEEC3C8
:106044009D5035EEC39F5030900776E0FC126CD41F
:106054003CF583E0FD9008F51244B68E827583000A
:10606400ED12420A900776126CBB126CEB700312AD
:106074006CDD126CB80E80C1EEC39F50149007768D
:10608400126CBB126CEB7003126CDD126CB80E80D8
:10609400E79007D0126CE443E6029008F8E0FEEFC4
:0860A400C39E50028002AF060A
:0160AC0022D1
:0C756D00126CC240047F0180027F0022EB
:03501800025452ED
:10545200C0E0C0F0C083C082C0D075D000C000C020
:0354620006C0077A
:10546500C218AFC1EF1244F6549B08549B1054ABBD
:105475001854B02054BD2854EA3054F53854FD6012
:1054850054F86854FD7054F87855048055049055C7
:1054950060A00000556E9007BEE0F5C2C2C590073A
:1054A500BDE4F00255709007BF802890077A74FD1F
:1054B500F0D2C4D2C50255709007BFE0FF9007BD7A
:1054C500E0C39F5014E0FF04F074C02FF582E4346C
:1054D50007F583E0F5C2025570D2C490077AE4F06F
:1054E500C210025570D2C590077A74FEF00255704D
:1054F500025565D20E025570900770E4F0806C90ED
:105505000770E07020E5C2F0E0FFC3900772E09FEE
:105515007480F8900771E0648098500312711090C0
:105525000770E004F0900771126CE490077B126C31
:10553500D23EF583E5C2F090077B126CBBFEE5F029
:1055450064404E700690077BF0A3F0900770E0145E
:10555500F070189007D0126CBC8010300E0DC20E82
:105565009007BDE4F0D2C58002D21830180EC2C62D
:0E557500D2C6C2C5C2C4D2C2C218C210C2C3BE
:10558300D007D006D000D0D0D082D083D0F0D0E0E6
:0155930032E5
:05760A00A2C7E433FFFC
:01760F002258
:106BB90074FFF5F00242937403F0A374E8F0A3E5BF
:106BC90084F0E4F58422D2C4D2C5D2C2C2C3E4900F
:106BD9000931F0FF22EFF0A3ECF0A3EDF0A302449A
:106BE900EDE5088509F0024293E025E044A0F5C2ED
:036BF9007F0322F5
:06761000C2C253E6FD2298
:065B5100900838126BDE23
:105B5700900841126BC020C7FDC2C4D2C2D2C5E4AF
:105B6700FF900931F030C3FDAEC1EE1244F65B91F0
:105B7700005B94085B94105BA2185BAC205BB428B5
:105B87005C07305C0F3800005B91025C17EF700612
:105B9700900838126BF2C2C5025C1D900839E0F517
:105BA700C27F0580719009317403F08069EFB405F5
:105BB7000B900839A3E0F5C27F06805AEF640670A0
:105BC7002D900840E090083B700875F0011244BF23
:105BD70080031244B61241B2F5C290083E126BB967
:105BE70090083EE07002A3E0702C7F078028EFB496
:105BF7000706D2C47F09801E9009317405F080160C
:105C07009009317404F0800E9009317406F0800613
:105C17009009317401F0EFB40904C2C380279009D9
:105C270031E0B4030D900841126BB945F0600312DF
:105C37006BCF900931E06008C2C5D2C4C2C38005EA
:0E5C4700C2C3025B6C20C7FD900843E0F584E9
:015C5500222C
:0657F500900850126BDE6B
:1057FB00900858126BC020C7FDD2C2C2C4D2C5E4F8
:10580B00FF900931F030C3FDAEC1EE1244F6583EA5
:10581B00005841085841105866185870205878287D
:10582B00589330589B3858A34058B35058DA580007
:10583B0000583E0258E0C2C5EF7009900850126B39
:10584B00F20258E6EF640160030258E6900850E05C
:10585B0025E044A1F5C27F040258E6900851E0F51B
:10586B00C27F0580769009317403F0806EEFB4052A
:10587B000B900851A3E0F5C27F06805FEFB40606DC
:10588B00D2C57F01805580189009317404F0804B8C
:10589B009009317406F08043EFB404047F02803B1F
:1058AB009009317405F08033900853E475F00112C0
:1058BB0044BFE5C21241F8900856126BB9900856D6
:1058CB00E07002A3E07004C2C280107F02800CD291
:1058DB00C47F0980069009317401F0EFB40904C24A
:1058EB00C38027900931E0B4030D900858126BB9AF
:1058FB0045F06003126BCF900931E06008C2C5D24E
:10590B00C4C2C38005C2C302581020C7FD90085AF9
:03591B00E0F58430
:01591E002266
:105A3A00900870EFF09008731244ED900871ECF042
:035A4A00A3EDF0D9
:105A4D00750A00543FF50B543F604BC37440950BE2
:105A5D00FFE4950AFE900876E0FCA3E0FDC39FEC01
:105A6D009E50068C088D0980048E088F09125B28C4
:105A7D0060037F0222900871126BEA900878E07043
:105A8D0006900874126BEAC3900877E09509F090C0
:105A9D000876E09508F0900876E0F508A3E0F509A2
:105AAD00D3E5099400E5089400406DE5099440E5BF
:105ABD00089400500F125B2860037F0222E4F50862
:105ACD00F50980DC900870E0FFA3E0FCA3E0FDA3E6
:105ADD001244B690083EE4F0A37440F0900878E0CC
:105AED00900840F0125B51900931E060037F022273
:105AFD0074C02509F50974FF3508F508900871E49F
:105B0D0075F040124293900878E070949008747587
:0A5B1D00F040124293025AAD7F00DF
:105B270022900870E0FFA3E0FCA3E0FDA31244B6B7
:105B370090083EE508F0A3E509F0900878E09008A2
:0A5B470040F0125B51900931E0229A
:10737200900856E4F0A304F01257F5900931E0604A
:07738200037F01227F0022BE
:10725D00900930EBF07B017A097930900876E4F0F3
:0A726D00A304F0E4A3F0125A3A2241
:10702800C007900888E0FFA3E0900856CFF0A3EFD0
:10703800F0D0071257F5900931E060037F01227FF5
:02704800002224
:10727700C007900890E0FFA3E0900876CFF0A3EF57
:0A728700F0E4A3F0D007125A3A22F7
:107291007B01E49008DDF0227422F0A3EFF0A32239
:0A72A1007B01E49008DDF07D04227B
:0B6C3E009008D91244ED9008DCEDF046
:106C4900E49008DEF09008D91244B69008DCE09090
:106C590008BCF09008DDE09008BDF0E4FF12661D65
:106C6900EFB4FF0D9008DEE0FE04F0EEC39403409C
:036C7900D47E00C6
:016C7C0022F5
:06704A0090090C1244ED58
:107050007E007F007D1012454990090C1244B67DD8
:0B70600010126009EF7002FF227F0198
:01706B002202
:106941009008661272997413F01241B2900869F0BE
:106951009000011241CB90086AF09000021241CBE5
:1069610090086BF09000031241CB90086CF09000FE
:10697100041241CB90086DF09000051241CB9008B4
:106981006EF09000061241CB90086FF07A0879669C
:086991001272917D0A026C3EB6
:1072F7009008F91272997403F0A374FFF07A087971
:09730700F91272917D04026C3E42
:107389009008FD127299741CF0A374FFF07A0879C1
:07739900FD1272A1026C3E1F
:10731000E4900901F0A3EFF0A3740AF0A3EFF07A70
:097320000979011272A1026C3E10
:0452B7004108270083
:10747A00E4F584900827F0F5BAF5BB75BCC075E849
:02748A0080225E
:03503000026764B0
:10676400C0E0C0F0C083C082C0D075D000C000C0FB
:1067740001C002C003C004C005C006C00775840080
:1067840053E8DF900827E025E02417F582E4340875
:10679400F583E5BFF0A3E5BEF0900827E004F0C35D
:1067A40094084005E4F0124E1C900827E0F5BBD095
:1067B40007D006D005D004D003D002D001D000D039
:0A67C400D0D082D083D0F0D0E032B4
:0F750000E4F58475D48075840175D480F58422F8
:1073B7007810E0FEA3E0A60608F62292AFAF028F90
:0673C700B1AF038F842228
:10682D00AB84AAB1A2AF921990090512445D9009EB
:10683D00071273B753B10F900906E0700543B110FD
:10684D008019900907E030E70543B130800D43B161
:10685D0020900907E04480F01273B7E4F584C2AFCD
:10686D0043B701758F037810E6FE08E6F5828E8337
:0C687D00E4F053B7FEF58FA2191273C2AD
:0168890022EC
:1065A700AB84AAB1A2AF921A90087E12445D9008FC
:1065B7007DE0F9FF3395E0FEEFF44E6053900880DD
:1065C70078121273B953B10F90087FE0700543B189
:1065D700108020900880E030E70543B130801443F5
:1065E700B120900880E04480F0E0FEA3E07812A696
:1065F7000608F6E4F584C2AF43B701758F01781238
:10660700E6FE08E6F5828E83E9F053B7FEE4F58FE0
:05661700A21A1273C27B
:01661C00225B
:1074F0000001FF00FF000001010000FF00FF01008C
:1052BB00032500002B032800002B410894F841081C
:1052CB0092F8C113C112410899004108930042089A
:1052DB00970000C111410895004108960001240078
:107329009400E09408900894E022E5288529838553
:097339002A822290090F0244B6D9
:104E1C00900894E0900892F0A2139212900817E078
:104E2C00FFA3E090089ECFF0A3EFF0E4FDFF125239
:104E3C00FEC390081BE094084004D2138002C213F6
:104E4C00A213B01250057F07126999D390081EE087
:104E5C0090081D12732940054408F0800354F7F0A4
:104E6C00D3900820E090081F12732940054410F0DD
:104E7C00800354EFF0D3900822E0940090082112A4
:104E8C00732B40054420F0800354DFF0D3900824AA
:104E9C00E0940090082312732B40054440F08003EB
:104EAC0054BFF0D3900826E0940090082512732B81
:104EBC0040054480F08003547FF0900894E0FC544B
:104ECC00187004A37403F0900892E0FE6CFDEE5D84
:104EDC00900921F0AF05EC5FA3F030E31890089532
:104EEC00E070047F01800B900895E054FEF0700593
:104EFC007F0A126999900921E030E5057F03126958
:104F0C0099900921E030E6057F04126999900921F6
:104F1C00E030E7057F05126999900899E0900893B5
:104F2C00F0A3E0F45410900899F0900895E0706AA2
:104F3C00900899E06033900893E07006900897F021
:104F4C00A3F0900897E475F001124293D39008985F
:104F5C00E09478900897E064809480403D20113A6A
:104F6C007F06126999D2118031900899E0702B90CC
:104F7C000893E06025900897E0FEA3E0FFD3940629
:104F8C00EE648094804011EF9478EE6480948050AD
:104F9C00077F02126999D211C211900922E030E404
:104FAC0010900895E0600A54FDF070057F0A1269B4
:014FBC00995B
:014FBD0022D1
:10699900AB25E5272401F9E43526FA90090F1244BD
:1069A900ED12733C90004BEB7008E965827003EAC5
:1069B9006583700BFB7A00792B90090F1244ED1255
:1069C900733C1273336B7008E965827003EA65835F
:1069D9006013AB25AA26A927EF1241F812733C8B45
:0569E900258A26892724
:0169EE002286
:106AE20053E6F7AB25AA26A9271273336525700A48
:106AF200E52765827004E52665837003FF802878A8
:106B020028E475F0011244A61241B2FF90004BE551
:106B120028700AE52A65827004E52965837008F504
:0A6B220028752900752A2B43E608A8
:016B2C002246
:106EFD0053E6F71273336525700AE5276582700432
:106F0D00E52665837003FF800AAB28AA29A92A12FA
:066F1D0041B2FF43E6084B
:016F2300224B
:0F750F00C3900823E0940840037F00227F0122ED
:03501E00025F62CC
:105F6200C0E0C0F0C083C082C0D075D000C001C004
:105F720002C003C005C006C007C2AF30DF02C2DFE5
:065F820020D90330D868AD
:105F8800E5905403900912F0C2D8C2D9900896E05F
:105F9800FF900912E0FD6F5403604D53E6F7EF756B
:105FA800F004A47E00540CFFED5403FDEF4D24F0E3
:105FB800F582EE3474F583E493FF900913F0A3E5BA
:105FC80024F0EF2524F524E0652430E1109009132E
:105FD800E0B401047F0880027F09126999900912D0
:085FE800E0900896F043E60882
:105FF000D2AFD007D006D005D003D002D001D0D088
:09600000D082D083D0F0D0E03250
:10668C00124451126B7590080B12445D900804E093
:10669C0025E0249EF582E43408F583E0FEA3E02295
:1066AC00FBC374FF9BFF740F9EFEE49400FDE49407
:1066BC0000FC22900804E025E0249AF582E43408DA
:1066CC0022900803E025E024C3F582E4340622E49A
:1066DC007F01FEFDFC124451C30243F7E47BFF7AB9
:0D66EC000FF9F82290080B1244510242DA17
:0852FE00900803EFF0A3EDF0AE
:105306001266C31266A5FBAA06E4F9F8126698FFB0
:10531600E4FCFD1242CC90080712445DE4900805B7
:10532600F0A3F07F0FFEFDFCA31266E14008900893
:1053360005E4F0A304F074FF7FF1FEFDFC9008077E
:10534600124451D31243F7500874FF900805F0A396
:10535600F0900805E0FEA3E0FF4E7003025451EF03
:07536600F47002EEF4705434
:10536D001266BF1266A5FFE4FCFD90081312445DA2
:10537D009008131266DB500A90081312446900005E
:10538D0000011266CD1266A5FFE4FCFD1266E9125E
:10539D0042DA90081312668CFFE4FCFD1266F09061
:1053AD00080F12445D1266E890080F124445126B07
:0153BD00757A
:0F53BE00025424900805E07004A3E064017064B9
:1053CD001266CD1266A51266AC1266E81242DA902C
:1053DD00080B12445D1266BF1266A51266AC9008EA
:1053ED000F12445D90080F1266DB500A90080F12E1
:1053FD0044690000000190080B12444590080F12FB
:10540D00668C1266AC1266F01266E8126B75C37488
:10541D00FF9FFF740F9EFE1266CDF583EEF0A3EF96
:04542D00F012501B0E
:10543100900804E0FF25E0249EF582E43408F5831A
:10544100E0FCA3E0FDEF1266C3F583ECF0A3EDF001
:015451002238
:10735A0000320078007D00830088009100A400B606
:08736A0000C800DB00EE00FF8B
:1073CD0033FE745A2FF58274733EF583740193C4A2
:0673DD00F8540FC86822FD
:1073A000E4F5B0F5A0F590F584F5D3F5D275840138
:0773B000F5D3F5D2F58422AC
:104C4A00E49008C3F0FF9006C5E0FCA3E0FBAA04C9
:104C5A009006B6E0FEB401057402FF8008EEB402C5
:104C6A0004EF4401FF9006B5E0FE7006EF4408FF2A
:104C7A008008EEB40104EF4404FF9006C0E014601B
:104C8A001014601314601624037016EF4410FF808A
:104C9A0010EF4420FF800AEF4440FF8004EF448075
:104CAA00FF8FB0C3EB9448EA940040089008C3749D
:104CBA003FF08058C3EB943CEA940040089008C344
:104CCA00749FF08047C3EB9430EA94004008900840
:104CDA00C374CFF08036C3EB9424EA940040089062
:104CEA0008C374E7F08025C3EB9418EA94004008DF
:104CFA009008C374F3F08014C3EB940CEA94009008
:104D0A0008C3400574F9F0800374FCF07C007D0C44
:104D1A00AF03AE0212423EED25E0FFEC1273CDFE68
:104D2A00E493C454F0489008C4F0A3CEF0AE04AFA4
:104D3A0005C3740B9FFFE49EFEEF25E0FFEE12739E
:104D4A00CDFFE493C454F048FEC3EB940CEA9400FC
:104D5A004008EB9418EA94004028C3EB9424EA94A0
:104D6A00004008EB9430EA94004017C3EB943CEA05
:104D7A0094004008EB9448EA94004006EB64544AD5
:104D8A0070139008C4E0FDA3E09008BFCDF0A3ED36
:104D9A00F0A3EE80139008BFEEF0A3EFF09008C4E2
:104DAA00E0FFA3E09008C1CFF0A3EFF075A0FFE405
:104DBA00F5849008BFE0FEA3E0FF8ED38FD27584FE
:104DCA0001A3E0FEA3E0FF8ED38FD2E4F584A3E033
:104DDA00F5A030030543901080035390EF9004260A
:104DEA00E014600C1460112402701353903F800E7B
:104DFA005390BF439080800653907F439040300C7D
:104E0A000543900480035390FB90041BE024FF9217
:014E1A009304
:014E1B002274
:0875E10018100C080604030257
:0652EB0041093200C11B65
:1074BF00F9F8126B759008E412445D9008E40244E9
:0174CF004577
:1070AE009000031241CB2406600D14601014600A88
:1070BE002404700C025D2502741F02755412752C87
:0170CE00229F
:10741F00D21BE4900932F09006B5E0B40204A374D5
:03742F0001F02247
:0D755400C21B9006B5E0B40203E4A3F022D0
:0E752C00D21B9006B5E0B40204A37401F02255
:105D2500201B03025DF3900932E0FF04F0EFB4603D
:0F5D3500037401F09006B5E064026003025DF3B1
:105D44009006C5A3E0FF75F00C1241909008E8F0AE
:105D54009006C3E0FEA3E0FFE42FFBEE34F8FAE480
:105D640034FFF9E434FFF8900819E0FEA3E0FFE4FF
:105D7400FCFD1242DA1274C4E4FB7A081274BFE424
:105D84007B2D7A021274BF9008E8E02FF0E0FFC385
:105D9400648094805004E4F0800ED3EF6480948790
:105DA40040069008E87407F09008E8E0FF3395E0B7
:105DB400FE74E12FF58274753EF583E493FD33950B
:105DC400E0FC900932E024FFFFE434FFFE12423E7F
:105DD400ED701C9006B6E064016011900426E0FFAB
:0F5DE40064016008EF6402600330060312496F28
:015DF300228D
:106E020075840F758A83E4F589F58475B7307584C6
:106E12000F438901758D01758E04758F017FFFDF28
:0C6E2200FE438902E58930E4FB7597020D
:016E2E002241
:0852F1004109240041092300DA
:0452F90041076F00FA
:1063A800900862E075F05D90D00112449AAF82AE19
:1063B8008322E475F001124293900864E475F001B9
:1063C8000242937A0679B57B019008B6E4F0A3748B
:1063D8005DF02290085EEEF0A3EFF0E4900864F020
:1063E800A3F022AFF0FEE0FCA3E0F5828C83E493F7
:1063F800FD22F074FAA3F0A3E4F0A32275F05DA4E3
:106408002401F974D035F0FA7BFF22EBF0AC07A237
:10641800AFE433A3F0C2AF22E475F0010242A9ED64
:0B642800FFAD04EDCFF0A3EFF0E42285
:06761600E490076FF02272
:0775F70090076F7401F02200
:10614F009009257401F0E4A3F01275D97ED07F0079
:10615F007A0979251261E17EDB7F447A097926126B
:10616F0061E1126F707E007F5D7D007B017A0679A1
:10617F00B5124549E49006B7F09006C0F09006B806
:10618F001263FA74FAF0A3E41263FA74FAF0E4906B
:10619F0006B6F09006B5F09006C1F0A3F0740812A1
:1061AF0063FDF0A3742AF0E4FFEF25E024C7F58226
:1061BF00E43406F583E4F0A3F074F92FF582E434A8
:1061CF0006F583E4F00FEFB419DF1275BB7F1E02E3
:0261DF006DD180
:0E61E1007B019008B6E4F0A304F0126D622278
:1072AB0090DB44E493F4600990D000E493640160B4
:0A72BB000312614FE49006B3F022C5
:056DD100900927EFF01E
:106DD6001275D9E4900928F0900927E0FFA3E0FE98
:106DE600C39F501575F05DEE1263AF1263CB126D43
:0C6DF60062900928E004F080DF026F705A
:106F960030021820141F90076FE0700C90041C74C8
:106FA6000AF09004577401F0D214222001077FBB27
:066FB600126B2DD2012236
:03501B00026F968B
:1070CF009006B3E0FFC3941E5014EF12640478B51A
:1070DF007C067D017E007F5D12416A12631BC21424
:0170EF00227E
:1071A3009006B3E0C3941E50121275D99006B31221
:0C71B30063AB1263CB126D62126F70228E
:0B75BB001271A3C214200202C20122C0
:0861EF00900845EDF0A3EBF070
:1061F700A3E004F090084AEFF0A3EBF0900845E025
:10620700FF90084AE0FED39F505E75F05DEE126383
:10621700AF90084CEEF0A3EFF090084B1263AB90F1
:10622700084EEEF0A3EFF0E4900848F0A3F09008D2
:106237004E12642090084C1263EB12653090084CA4
:106247001263C49008481263C4C3900849E0945D80
:10625700900848E0940040D6126F7090084AE00416
:10626700F0A3E004F00262039006B3E0FF90084653
:0E627700E0D39F5009A3E0C39F40031270CFF5
:0162850022F6
:0F591F0090085CEDF090085BEFF090085DEBF006
:10592E00900862EFF0A3EBF090085CE0FF90086245
:10593E00E0D39F40030259F5A31263AB1263DB90D1
:10594E000864E0FEA3E0FFC3945DEE9400501A904D
:10595E00085E1263EE74122FF582E43407F583EDC0
:10596E00F090085E1263BA80D61263A8900860EEBB
:10597E00F0A3EFF09008631263AB1263DB90085E46
:10598E001264209008601263EB126530900860126A
:10599E0063BAC3900865E0945D900864E09400409B
:1059AE00DC1263A89008601263DE900864E0FCA32A
:1059BE00E0FDC3945DEC9400501D900860126420CD
:1059CE00AFF0FE74122DF582E43407F583E0FD127C
:1059DE0065301263C180D3126F70900862E004F0DC
:1059EE00A3E004F00259369006B3E0FF90085DE0A4
:1059FE00FED39F502090085BE0FDA3E0C39DFDE425
:105A0E009400FCEE7A002DFDEA3CFCC3ED9F748001
:105A1E00F86C9850139006B3E0FF90085BE0D39FAC
:0B5A2E005009A3E0C39F40031270CF9B
:015A3900224A
:0364B5009008A2AA
:1064B8001264131276109008A81264279008A4F0AA
:1064C8009008A2E0FF9008A8E0FCA3E0FD7B017A19
:1064D8000779129008881263D41270289008A8E4EB
:1064E80075F05D1242939008A4E0126404A312446C
:1064F800ED1275D99008A51244B6AE02AF017A071D
:1065080079121263CF126D62126F709008A4E004C2
:10651800F0E0C3941E40A99004A5E0FF12754790CF
:0765280008A3E024FF92AF7D
:01652F002249
:0366F9009008C640
:1066FC001264131276109008C91264279008C8F01F
:10670C009008C8E0FFC3941E503D75F05DEF126316
:10671C00AF9008CBEEF0FAA3EFF0FB9008C6E0FFC9
:10672C009008C9E0FCA3E0FDA9037BFF9008901240
:10673C0063D41272779008C9E475F05D124293909D
:10674C0008C8E004F080B99004A5E0FF12754790EA
:07675C0008C7E024FF92AF23
:016763002213
:03000000024000BB
:03000300025003A5
:03000B000250069A
:030013000250098F
:03001B0002500C84
:0300230002500F79
:03002B000250126E
:0300330002501563
:03003B0002501858
:0300430002501B4D
:03004B0002501E42
:0300530002502137
:03005B000250242C
:0300630002502721
:03006B0002502A16
:0300730002502D0B
:03007B0002503000
:03008300025033F5
:03008B00025036EA
:03009300025039DF
:03009B0002503CD4
:0300A30002503FC9
:10400000787FE4F6D8FD9000007F007E20E4F0A3E6
:0A401000DFFCDEFA75814A0240551C
:10401A00024575E493A3F8E493A34003F68001F202
:10402A0008DFF48029E493A3F85407240CC8C333A7
:10403A00C4540F4420C8834004F456800146F6DF76
:10404A00E4800B01020408102040809051A8E47E0D
:10405A00019360BCA3FF543F30E509541FFEE4936B
:10406A00A360010ECF54C025E060A840B8E493A332
:10407A00FAE493A3F8E493A3C8C582C8CAC583CA5D
:10408A00F0A3C8C582C8CAC583CADFE9DEE780BE15
:0152FD0000B0
:10409A00E709F608DFFA8046E709F208DFFA803E08
:1040AA0088828C83E709F0A3DFFA8032E309F608F5
:1040BA00DFFA8078E309F208DFFA807088828C835D
:1040CA00E309F0A3DFFA806489828A83E0A3F60811
:1040DA00DFFA805889828A83E0A3F208DFFA804CEB
:1040EA0080D280FA80C680D4806980F280338010C2
:1040FA0080A680EA809A80A880DA80E280CA80332B
:10410A0089828A83ECFAE493A3C8C582C8CCC583A2
:10411A00CCF0A3C8C582C8CCC583CCDFE9DEE78072
:10412A000D89828A83E493A3F608DFF9ECFAA9F0F1
:10413A00EDFB2289828A83ECFAE0A3C8C582C8CC47
:10414A00C583CCF0A3C8C582C8CCC583CCDFEADE60
:10415A00E880DB89828A83E493A3F208DFF980CCC2
:10416A0088F0EF60010E4E60C388F0ED2402B404BB
:10417A000050B9F582EB2402B4040050AF23234562
:06418A0082239040EA735D
:10419000C2D530F707B2D563F0FF05F030E70CB2B7
:1041A000D5F4048463F0FF05F080018430D502F477
:0241B0000422E7
:1041B200BB010689828A83E0225002E722BBFE020B
:0941C200E32289828A83E493223E
:1041CB00BB010CE58229F582E5833AF583E02250A9
:1041DB0006E92582F8E622BBFE06E92582F8E222F3
:0D41EB00E58229F582E5833AF583E493220D
:1041F800BB010689828A83F0225002F722BBFE01A6
:02420800F3229F
:10420A00F8BB010DE58229F582E5833AF583E8F0EA
:10421A00225006E92582C8F622BBFE05E92582C896
:02422A00F2227E
:10422C00EF8DF0A4A8F0CF8CF0A428CE8DF0A42EA6
:02423C00FE2260
:10423E00BC000BBE0029EF8DF084FFADF022E4CC64
:10424E00F875F008EF2FFFEE33FEEC33FCEE9DEC2D
:10425E00984005FCEE9DFE0FD5F0E9E4CEFD22ED73
:10426E00F8F5F0EE8420D21CFEADF075F008EF2FBD
:10427E00FFED33FD4007985006D5F0F222C398FDAE
:05428E000FD5F0EA224B
:10429300C5F0F8A3E028F0C5F0F8E58215827002B6
:0642A3001583E038F02253
:1042A900A3F8E0C5F025F0F0E582158270021583C8
:0642B900E0C838F0E82225
:0D42BF00EF2BFFEE3AFEED39FDEC38FC224E
:0E42CC00C3EF9BFFEE9AFEED99FDEC98FC22ED
:1042DA00E88FF0A4CC8BF0A42CFCE98EF0A42CFC83
:1042EA008AF0EDA42CFCEA8EF0A4CDA8F08BF0A401
:1042FA002DCC3825F0FDE98FF0A42CCD35F0FCEB60
:10430A008EF0A4FEA9F0EB8FF0A4CFC5F02ECD3924
:0F431A00FEE43CFCEAA42DCE35F0FDE43CFC2291
:1043290075F008758200EF2FFFEE33FECD33CDCC4B
:1043390033CCC58233C5829BED9AEC99E5829840CE
:104349000CF582EE9BFEED9AFDEC99FC0FD5F0D6AB
:10435900E4CEFBE4CDFAE4CCF9A88222B800C1B9D5
:104369000059BA002DEC8BF084CFCECDFCE5F0CB13
:10437900F97818EF2FFFEE33FEED33FDEC33FCEB4C
:1043890033FB10D703994004EB99FB0FD8E5E4F907
:10439900FA227818EF2FFFEE33FEED33FDEC33FCF4
:1043A900C933C910D7059BE99A4007EC9BFCE99AE8
:1043B900F90FD8E0E4C9FAE4CCFB2275F010EF2F2D
:1043C900FFEE33FEED33FDCC33CCC833C810D7072D
:1043D9009BEC9AE899400AED9BFDEC9AFCE899F868
:0E43E9000FD5F0DAE4CDFBE4CCFAE4C8F922FB
:106B7500C2D5E830E70FB2D5E4C39BFBE49AFAE44B
:106B850099F9E498F8EC30E717B2D5126BAB1243DC
:106B950065E4C39BFBE49AFAE499F9E498F8800369
:106BA50012436530D50DE4C39FFFE49EFEE49DFDD1
:046BB500E49CFC223E
:1043F700EB9FF5F0EA9E42F0E99D42F0EC6480C83D
:0644070064809845F022DC
:10440D00EB9FF5F0EA9E42F0E99D42F0E89C45F005
:01441D00227C
:10441E00E8600FECC313FCED13FDEE13FEEF13FF7C
:03442E00D8F122A0
:10443100E86010ECA2E713FCED13FDEE13FEEF13A1
:04444100FFD8F0228E
:0C444500E0FCA3E0FDA3E0FEA3E0FF22EA
:0C445100E0F8A3E0F9A3E0FAA3E0FB22EE
:0C445D00ECF0A3EDF0A3EEF0A3EFF022D2
:10446900A8828583F0D083D08212448012448012BE
:104479004480124480E473E493A3C583C5F0C583E3
:10448900C8C582C8F0A3C583C5F0C583C8C582C89D
:014499002200
:0C449A00A42582F582E5F03583F583222D
:1044A600FAE6FB0808E6F925F0F618E6CA3AF62217
:0944B600E0FBA3E0FAA3E0F92207
:1044BF00F8E0FBA3A3E0F925F0F0E5821582700286
:0744CF001583E0FA38F0222A
:1044D600F8E0FBA3A3E025F0F9F0E582158270026F
:0744E6001583E038FAF02213
:0944ED00EBF0A3EAF0A3E9F022D0
:1044F600D083D082F8E4937012740193700DA3A355
:1045060093F8740193F5828883E473740293686068
:06451600EFA3A3A380DF68
:10451C00EC8EF0A4CCC5F0CCCDF8EFA4CEC5F02D2C
:10452C00FDE43CFCE8A42EC8C5F03DFDE43CFCEFEA
:0D453C00A4FFE5F028FEE43DFDE43CFC2278
:10454900EF4E6012EF60010EEDBB010B89828A8389
:10455900F0A3DFFCDEFA2289F05007F709DFFCA996
:0C456900F022BBFEFCF309DFFCA9F022ED
:00000001FF
